 sim

 Timestamp is 4fb04cc2 (Mon May 14 12:07:30 2012)

 Preferred load address is 10000000

 Start         Length     Name                   Class
 0001:00000000 000007d6H .rdata                  CODE
 0001:000007d8 00000020H .rdata$debug            CODE
 0001:000007f8 000044b0H .text                   CODE
 0001:00004ca8 00000028H .xdata                  CODE
 0001:00004cd0 0000003cH .idata$2                CODE
 0001:00004d0c 00000014H .idata$3                CODE
 0001:00004d20 000000d8H .idata$4                CODE
 0001:00004df8 000000a2H .idata$6                CODE
 0001:00004ea0 000000ffH .edata                  CODE
 0002:00000000 000000d8H .idata$5                DATA
 0002:000000d8 00000328H .data                   DATA
 0002:00000400 00000048H .bss                    DATA
 0003:00000000 000001e0H .pdata                  DATA

  Address         Publics by Value              Rva+Base       Lib:Object

 0000:00000000       ___safe_se_handler_count   00000000     <absolute>
 0000:00000000       ___safe_se_handler_table   00000000     <absolute>
 0001:000000b0       ??_C@_19OBNDINH@?$AAP?$AAo?$AAr?$AAt?$AA?$AA@ 100010b0     sim_common_topaz_v1:simce.obj
 0001:000000bc       ??_C@_1CC@KMPFMANC@?$AAD?$AAe?$AAv?$AAi?$AAc?$AAe?$AAA?$AAr?$AAr?$AAa?$AAy?$AAI?$AAn?$AAd?$AAe?$AAx?$AA?$AA@ 100010bc     sim_common_topaz_v1:simce.obj
 0001:000000e0       ??_C@_19DINFBLAK@?$AAN?$AAa?$AAm?$AAe?$AA?$AA@ 100010e0     sim_common_topaz_v1:simce.obj
 0001:000000ec       ??_C@_19GFKPKJIA@?$AA?5?$AA?$FL?$AA?5?$AA?$FN?$AA?$AA@ 100010ec     sim_common_topaz_v1:simce.obj
 0001:000000f8       ??_C@_09JJPIIJJC@Freescale?$AA@ 100010f8     sim_common_topaz_v1:simce.obj
 0001:00000188       NTStatusC000Table          10001188     smclib:smcce.obj
 0001:00000718       NTStatus8000Table          10001718     smclib:smcce.obj
 0001:00000768       ??_C@_1CM@MEAEFIBF@?$AAS?$AAC?$AAa?$AAr?$AAd?$AAI?$AAn?$AAt?$AAr?$AAo?$AAd?$AAu?$AAc?$AAe?$AAR?$AAe?$AAa?$AAd?$AAe?$AAr?$AAW?$AA?$AA@ 10001768     smclib:smcce.obj
 0001:00000794       ??_C@_1CG@HNJJIDPF@?$AAS?$AAC?$AAa?$AAr?$AAd?$AAF?$AAo?$AAr?$AAg?$AAe?$AAt?$AAR?$AAe?$AAa?$AAd?$AAe?$AAr?$AAW?$AA?$AA@ 10001794     smclib:smcce.obj
 0001:000007bc       ??_C@_1BK@JIMBCHBC@?$AAW?$AAI?$AAN?$AAS?$AAC?$AAA?$AAR?$AAD?$AA?4?$AAD?$AAL?$AAL?$AA?$AA@ 100017bc     smclib:smcce.obj
 0001:000007f8       BSPGetSIMCLK               100017f8 f   bspsim.obj
 0001:00000840       BSPSetSIMClockGatingMode   10001840 f   bspsim.obj
 0001:000008ac       BSPSimIomuxSetPin          100018ac f   bspsim.obj
 0001:00000b24       BSPSimSelect3Volts         10001b24 f   bspsim.obj
 0001:00000b94       DllEntry                   10001b94 f   sim_common_topaz_v1:simce.obj
 0001:00000cd8       SCR_Open                   10001cd8 f   sim_common_topaz_v1:simce.obj
 0001:00000dcc       SCR_Close                  10001dcc f   sim_common_topaz_v1:simce.obj
 0001:00000ec0       SCR_IOControl              10001ec0 f   sim_common_topaz_v1:simce.obj
 0001:00000f5c       SCR_Read                   10001f5c f   sim_common_topaz_v1:simce.obj
 0001:00000f64       SCR_Write                  10001f64 f   sim_common_topaz_v1:simce.obj
 0001:00000f6c       SCR_Seek                   10001f6c f   sim_common_topaz_v1:simce.obj
 0001:00000f74       SCR_PowerUp                10001f74 f   sim_common_topaz_v1:simce.obj
 0001:00000f78       SCR_PowerDown              10001f78 f   sim_common_topaz_v1:simce.obj
 0001:000011f4       SCR_Deinit                 100021f4 f   sim_common_topaz_v1:simce.obj
 0001:000014a8       SCR_Init                   100024a8 f   sim_common_topaz_v1:simce.obj
 0001:00001520       CBCardPower                10002520 f   sim_common_topaz_v1:simcb.obj
 0001:00001800       CBCardTracking             10002800 f   sim_common_topaz_v1:simcb.obj
 0001:00001818       CBUpdateCardState          10002818 f   sim_common_topaz_v1:simcb.obj
 0001:00001864       CBSetProtocol              10002864 f   sim_common_topaz_v1:simcb.obj
 0001:00001a70       CBTransmit                 10002a70 f   sim_common_topaz_v1:simcb.obj
 0001:00001aec       SIM_InternalMapRegisterAddresses 10002aec f   sim_common_topaz_v1:simhw.obj
 0001:00001b08       SIM_InternalUnMapRegisterAddresses 10002b08 f   sim_common_topaz_v1:simhw.obj
 0001:00001b20       SIM_Close                  10002b20 f   sim_common_topaz_v1:simhw.obj
 0001:00001bd8       SIM_ColdReset              10002bd8 f   sim_common_topaz_v1:simhw.obj
 0001:000021a8       SIM_WarmReset              100031a8 f   sim_common_topaz_v1:simhw.obj
 0001:00002314       SIM_ReadData               10003314 f   sim_common_topaz_v1:simhw.obj
 0001:00002454       SIM_WriteData              10003454 f   sim_common_topaz_v1:simhw.obj
 0001:00002518       SIM_Deactivate             10003518 f   sim_common_topaz_v1:simhw.obj
 0001:000025b0       SIM_ConfigCLK              100035b0 f   sim_common_topaz_v1:simhw.obj
 0001:000027a4       SIM_ConfigTime             100037a4 f   sim_common_topaz_v1:simhw.obj
 0001:000027e0       SIM_CheckCard              100037e0 f   sim_common_topaz_v1:simhw.obj
 0001:00002804       SIM_FlushFIFO              10003804 f   sim_common_topaz_v1:simhw.obj
 0001:0000284c       SIM_Init                   1000384c f   sim_common_topaz_v1:simhw.obj
 0001:00002b0c       LeaveCriticalSection       10003b0c f   coredll:COREDLL.dll
 0001:00002b1c       EnterCriticalSection       10003b1c f   coredll:COREDLL.dll
 0001:00002b2c       InterlockedIncrement       10003b2c f   coredll:COREDLL.dll
 0001:00002b3c       DeleteCriticalSection      10003b3c f   coredll:COREDLL.dll
 0001:00002b4c       DisableThreadLibraryCalls  10003b4c f   coredll:COREDLL.dll
 0001:00002b5c       InitializeCriticalSection  10003b5c f   coredll:COREDLL.dll
 0001:00002b6c       Sleep                      10003b6c f   coredll:COREDLL.dll
 0001:00002b7c       StringCchCopyW             10003b7c f   coredll:COREDLL.dll
 0001:00002b8c       InterlockedDecrement       10003b8c f   coredll:COREDLL.dll
 0001:00002b9c       CreateThread               10003b9c f   coredll:COREDLL.dll
 0001:00002bac       SetLastError               10003bac f   coredll:COREDLL.dll
 0001:00002bbc       CloseHandle                10003bbc f   coredll:COREDLL.dll
 0001:00002bcc       WaitForSingleObject        10003bcc f   coredll:COREDLL.dll
 0001:00002bdc       RegCloseKey                10003bdc f   coredll:COREDLL.dll
 0001:00002bec       RegQueryValueExW           10003bec f   coredll:COREDLL.dll
 0001:00002bfc       OpenDeviceKey              10003bfc f   coredll:COREDLL.dll
 0001:00002c0c       RegOpenKeyExW              10003c0c f   coredll:COREDLL.dll
 0001:00002c1c       StringCchCatW              10003c1c f   coredll:COREDLL.dll
 0001:00002c2c       LocalFree                  10003c2c f   coredll:COREDLL.dll
 0001:00002c3c       LocalAlloc                 10003c3c f   coredll:COREDLL.dll
 0001:00002c4c       EventModify                10003c4c f   coredll:COREDLL.dll
 0001:00002c5c       KernelIoControl            10003c5c f   coredll:COREDLL.dll
 0001:00002c6c       InterruptDisable           10003c6c f   coredll:COREDLL.dll
 0001:00002c7c       InterruptDone              10003c7c f   coredll:COREDLL.dll
 0001:00002c8c       InterruptInitialize        10003c8c f   coredll:COREDLL.dll
 0001:00002c9c       CreateEventW               10003c9c f   coredll:COREDLL.dll
 0001:00002cac       MmMapIoSpace               10003cac f   ceddk:CEDDK.dll
 0001:00002cbc       MmUnmapIoSpace             10003cbc f   ceddk:CEDDK.dll
 0001:00002ccc       DDKClockGetFreq            10003ccc f   cspddk:CSPDDK.dll
 0001:00002cdc       DDKClockSetGatingMode      10003cdc f   cspddk:CSPDDK.dll
 0001:00002cec       DDKGpioWriteDataPin        10003cec f   cspddk:CSPDDK.dll
 0001:00002cfc       DDKGpioSetConfig           10003cfc f   cspddk:CSPDDK.dll
 0001:00002d0c       DDKIomuxSetPadConfig       10003d0c f   cspddk:CSPDDK.dll
 0001:00002d1c       DDKIomuxSetPinMux          10003d1c f   cspddk:CSPDDK.dll
 0001:00002d2c       SmartcardCreateLink        10003d2c f   smclib:smcce.obj
 0001:00002dc8       SmartcardDeleteLink        10003dc8 f   smclib:smcce.obj
 0001:00002e08       SmartcardInitialize        10003e08 f   smclib:smcce.obj
 0001:00002f78       SmartcardExit              10003f78 f   smclib:smcce.obj
 0001:00003054       SmartcardCompleteCardTracking 10004054 f   smclib:smcce.obj
 0001:00003070       MapNtStatusToWinError      10004070 f   smclib:smcce.obj
 0001:000030e0       SmartcardDeviceControl     100040e0 f   smclib:smcce.obj
 0001:00003420       SmartcardInitializeCardCapabilities 10004420 f   smclib:smcutil.obj
 0001:0000348c       SmartcardInvertData        1000448c f   smclib:smcutil.obj
 0001:00003500       SmartcardUpdateCardCapabilities 10004500 f   smclib:smcutil.obj
 0001:00003dec       SmartcardT0Request         10004dec f   smclib:smcprot.obj
 0001:00003ef4       SmartcardT0Reply           10004ef4 f   smclib:smcprot.obj
 0001:00003f80       SMCDeviceIoControl         10004f80 f   smclib:smcioctl.obj
 0001:00004a6c       __GSHandlerCheckCommon     10005a6c f   corelib0:gshandler.obj
 0001:00004aa8       __GSHandlerCheck           10005aa8 f   corelib0:gshandler.obj
 0001:00004acc       __security_check_cookie    10005acc f   corelib0:armsecgs.obj
 0001:00004ae0       __gsfailure                10005ae0 f   corelib0:armsecgs.obj
 0001:00004b24       wcslen                     10005b24 f   corelib1:COREDLL.dll
 0001:00004b34       memset                     10005b34 f   corelib1:COREDLL.dll
 0001:00004b44       mbstowcs                   10005b44 f   corelib1:COREDLL.dll
 0001:00004b54       memcpy                     10005b54 f   corelib1:COREDLL.dll
 0001:00004b64       memcmp                     10005b64 f   corelib1:COREDLL.dll
 0001:00004b74       __rt_sdiv                  10005b74 f   corelib1:COREDLL.dll
 0001:00004b84       __C_specific_handler       10005b84 f   corelib1:COREDLL.dll
 0001:00004b94       __report_gsfailure         10005b94 f   corelib1:COREDLL.dll
 0001:00004ba4       CspSIMGetIRQs              10005ba4 f   sim_mx25_topaz_v1:cspsim.obj
 0001:00004c00       CspSIMGetBaseAddress       10005c00 f   sim_mx25_topaz_v1:cspsim.obj
 0001:00004c28       GetProcAddressW            10005c28 f   coredll:COREDLL.dll
 0001:00004c38       GetModuleHandleW           10005c38 f   coredll:COREDLL.dll
 0001:00004c48       CloseMsgQueue              10005c48 f   coredll:COREDLL.dll
 0001:00004c58       StopPowerNotifications     10005c58 f   coredll:COREDLL.dll
 0001:00004c68       ReadMsgQueue               10005c68 f   coredll:COREDLL.dll
 0001:00004c78       WaitForMultipleObjects     10005c78 f   coredll:COREDLL.dll
 0001:00004c88       RequestPowerNotifications  10005c88 f   coredll:COREDLL.dll
 0001:00004c98       CreateMsgQueue             10005c98 f   coredll:COREDLL.dll
 0001:00004cd0       __IMPORT_DESCRIPTOR_COREDLL 10005cd0     coredll:COREDLL.dll
 0001:00004ce4       __IMPORT_DESCRIPTOR_CEDDK  10005ce4     ceddk:CEDDK.dll
 0001:00004cf8       __IMPORT_DESCRIPTOR_CSPDDK 10005cf8     cspddk:CSPDDK.dll
 0001:00004d0c       __NULL_IMPORT_DESCRIPTOR   10005d0c     coredll:COREDLL.dll
 0002:00000000       __imp_MmMapIoSpace         10006000     ceddk:CEDDK.dll
 0002:00000004       __imp_MmUnmapIoSpace       10006004     ceddk:CEDDK.dll
 0002:00000008       \177CEDDK_NULL_THUNK_DATA  10006008     ceddk:CEDDK.dll
 0002:0000000c       __imp_DeleteCriticalSection 1000600c     coredll:COREDLL.dll
 0002:00000010       __imp_DisableThreadLibraryCalls 10006010     coredll:COREDLL.dll
 0002:00000014       __imp_InitializeCriticalSection 10006014     coredll:COREDLL.dll
 0002:00000018       __imp_Sleep                10006018     coredll:COREDLL.dll
 0002:0000001c       __imp_StringCchCopyW       1000601c     coredll:COREDLL.dll
 0002:00000020       __imp_InterlockedDecrement 10006020     coredll:COREDLL.dll
 0002:00000024       __imp_CreateThread         10006024     coredll:COREDLL.dll
 0002:00000028       __imp_SetLastError         10006028     coredll:COREDLL.dll
 0002:0000002c       __imp_CloseHandle          1000602c     coredll:COREDLL.dll
 0002:00000030       __imp_WaitForSingleObject  10006030     coredll:COREDLL.dll
 0002:00000034       __imp_RegCloseKey          10006034     coredll:COREDLL.dll
 0002:00000038       __imp_RegQueryValueExW     10006038     coredll:COREDLL.dll
 0002:0000003c       __imp_InterlockedIncrement 1000603c     coredll:COREDLL.dll
 0002:00000040       __imp_RegOpenKeyExW        10006040     coredll:COREDLL.dll
 0002:00000044       __imp_StringCchCatW        10006044     coredll:COREDLL.dll
 0002:00000048       __imp_LocalFree            10006048     coredll:COREDLL.dll
 0002:0000004c       __imp_LocalAlloc           1000604c     coredll:COREDLL.dll
 0002:00000050       __imp_EventModify          10006050     coredll:COREDLL.dll
 0002:00000054       __imp_KernelIoControl      10006054     coredll:COREDLL.dll
 0002:00000058       __imp_InterruptDisable     10006058     coredll:COREDLL.dll
 0002:0000005c       __imp_InterruptDone        1000605c     coredll:COREDLL.dll
 0002:00000060       __imp_InterruptInitialize  10006060     coredll:COREDLL.dll
 0002:00000064       __imp_CreateEventW         10006064     coredll:COREDLL.dll
 0002:00000068       __imp_LeaveCriticalSection 10006068     coredll:COREDLL.dll
 0002:0000006c       __imp_EnterCriticalSection 1000606c     coredll:COREDLL.dll
 0002:00000070       __imp_OpenDeviceKey        10006070     coredll:COREDLL.dll
 0002:00000074       __imp_RequestPowerNotifications 10006074     coredll:COREDLL.dll
 0002:00000078       __imp_WaitForMultipleObjects 10006078     coredll:COREDLL.dll
 0002:0000007c       __imp_ReadMsgQueue         1000607c     coredll:COREDLL.dll
 0002:00000080       __imp_StopPowerNotifications 10006080     coredll:COREDLL.dll
 0002:00000084       __imp_CloseMsgQueue        10006084     coredll:COREDLL.dll
 0002:00000088       __imp_GetModuleHandleW     10006088     coredll:COREDLL.dll
 0002:0000008c       __imp_GetProcAddressW      1000608c     coredll:COREDLL.dll
 0002:00000090       __imp_wcslen               10006090     corelib1:COREDLL.dll
 0002:00000094       __imp_memset               10006094     corelib1:COREDLL.dll
 0002:00000098       __imp_mbstowcs             10006098     corelib1:COREDLL.dll
 0002:0000009c       __imp_memcpy               1000609c     corelib1:COREDLL.dll
 0002:000000a0       __imp_memcmp               100060a0     corelib1:COREDLL.dll
 0002:000000a4       __imp___rt_sdiv            100060a4     corelib1:COREDLL.dll
 0002:000000a8       __imp___C_specific_handler 100060a8     corelib1:COREDLL.dll
 0002:000000ac       __imp___rt_udiv            100060ac     corelib1:COREDLL.dll
 0002:000000b0       __imp___report_gsfailure   100060b0     corelib1:COREDLL.dll
 0002:000000b4       __imp_CreateMsgQueue       100060b4     coredll:COREDLL.dll
 0002:000000b8       \177COREDLL_NULL_THUNK_DATA 100060b8     coredll:COREDLL.dll
 0002:000000bc       __imp_DDKIomuxSetPadConfig 100060bc     cspddk:CSPDDK.dll
 0002:000000c0       __imp_DDKGpioSetConfig     100060c0     cspddk:CSPDDK.dll
 0002:000000c4       __imp_DDKGpioWriteDataPin  100060c4     cspddk:CSPDDK.dll
 0002:000000c8       __imp_DDKClockSetGatingMode 100060c8     cspddk:CSPDDK.dll
 0002:000000cc       __imp_DDKClockGetFreq      100060cc     cspddk:CSPDDK.dll
 0002:000000d0       __imp_DDKIomuxSetPinMux    100060d0     cspddk:CSPDDK.dll
 0002:000000d4       \177CSPDDK_NULL_THUNK_DATA 100060d4     cspddk:CSPDDK.dll
 0002:000003f8       __security_cookie          100063f8     corelib0:seccinit.obj
 0002:000003fc       __security_cookie_complement 100063fc     corelib0:seccinit.obj
 0002:00000404       g_pfnIntroduceReader       10006404     smclib:smcce.obj
 0002:00000408       g_pfnForgetReader          10006408     smclib:smcce.obj
 0002:00000420       g_DriverCritSect           10006420     <common>
 0002:00000438       g_DeviceSlot               10006438     <common>
 0002:00000440       g_hReEnumerationEvent      10006440     <common>
 0002:00000444       g_IsResumed                10006444     <common>

 entry point at        0001:00000b94

 Static symbols

 0001:00000b28       ValidateAndEnterDevice     10001b28 f   sim_common_topaz_v1:simce.obj
 0001:00000bec       SIMCardDetectionThread     10001bec f   sim_common_topaz_v1:simce.obj
 0001:00000c74       SIMVendorIoctl             10001c74 f   sim_common_topaz_v1:simce.obj
 0001:00000f7c       GetIOIndex                 10001f7c f   sim_common_topaz_v1:simce.obj
 0001:0000104c       MakeFriendlyName           1000204c f   sim_common_topaz_v1:simce.obj
 0001:000010f4       SIMUnloadDevice            100020f4 f   sim_common_topaz_v1:simce.obj
 0001:00001210       SIMLoadDevice              10002210 f   sim_common_topaz_v1:simce.obj
 0001:0000164c       T0_ExchangeData            1000264c f   sim_common_topaz_v1:simcb.obj
